:03000000020C00EF
:03000300021A03DB
:03000B00021A06D0
:03001300021A09C5
:03001B00021A0CBA
:03002300021A0FAF
:03002B00021A12A4
:03003300021A1599
:03003B00021A188E
:03004300021A1B83
:03004B00021A1E78
:03005300021A216D
:03005B00021A2462
:03006300021A2757
:03006B00021A2A4C
:03007300021A2D41
:03007B00021A3036
:03008300021A332B
:03008B00021A3620
:03009300021A3915
:03009B00021A3C0A
:0300A300021A3FFF
:100C0000787FE4F6D8FD9000007F007E20E4F0A31A
:0A0C1000DFFCDEFA758176020C5558
:10335300C112C114C10F41152E0042152B0000C12B
:1033630093C18E4314F001146A4314F301146A44A5
:1033730014F7FFFFFFFFC11141152D004114EAFFB0
:10370900EFFD3395E0FC74F72DF58274143CF583D5
:103719002290135412182F89828A832290128CE0E6
:10372900D36480F8EE64809822EEFD3395E0FC7452
:10373900EC2DF58274143CF58322FE75F02DEF1201
:10374900181AE5822EF582E43583F5837401F09029
:103759000AD1E004F02274002FF582E43406F583DF
:1037690022900AD1E025E02416F582E43405F58398
:103779002290152AE0FF901602E06F22900AD1E00C
:10378900FF24DEF582E43405F58322EDFF3395E06D
:10379900FEEF25E0FFEE33FE22FBEAC4F854F0C841
:1037A900EBC4540F48900D71F022E475F001021436
:1037B900FF125B44EE547FFF22900AD1E0FFC3223F
:1037C900744F2FF582E43414F583223EF583EAF031
:1037D900A3EBF0223EF583E0FAA3E022901603E082
:1037E900FFA3E0FDA3E0FB22EC25E02424F8E6FAA0
:1037F90008E62290152B7427F0A37410F022901478
:10380900F002182F7B017A14796A02184F9014F389
:0938190002182F12182F0218AA40
:1061E40075840F75A4357580C075A57C75A7FF757A
:0661F400E11775E34422EF
:0F631900E4F584759A4075F809759D04C2FA225F
:105E6F00E4F584758850758921F58EF58D75C9080F
:105E7F0075CDFF75CCC075CBFF75CAE075C804F53D
:025E8F0084226B
:10628D00E4F584759105759852758401759810F52E
:02629D00842259
:10541700E4FFFE75840F438A0353A1DFF58475B754
:105427003075840F43A120438901758D01758F0164
:10543700758E040FBF00010EEF640F4E70F54389A0
:1054470002E58920E4130FBF00010EBE0FF3BFFF73
:0D545700F0E4F58443EF1080E87597022221
:0D63800075A89275B81075E60875E7402203
:10629F00E4F58475D84075D98375DA3175DB31D261
:0262AF00DE22ED
:106210001261E4125417125E6F12629F12628D12A5
:05622000631902638018
:0A63E0007F021261CD7F040261CD3F
:103FD300AC07E4900D72F0ED4430900D70F0E4FD09
:103FE300EDFF3395E0FE74FC2FF58274053EF583F7
:103FF300E06C7058900D7204F0ED12379674952FA3
:10400300F58274021237DD1237A2EB540FF912371F
:104013009474D92FF58274011237DDFB74952FF553
:104023008274021237D474F02FF58274001237DDD4
:10403300FB74D92FF58274011237D41237F1FB12B6
:10404300379474F02FF58274001237D40DED6404A5
:10405300708E900D72E0700C1237F11237A2AF031D
:10406300EF540FF9E9C454F0F9E59A20E7FBE4F5BE
:104073009BE59A20E7FB900D70E0F59BE59A20E71E
:10408300FB900D71E0F59BE59A20E7FB899BE59A90
:0440930020E7FB2205
:10436100900D6EEFF0121884438500439201439F34
:104371000243AC0343B90443C60543D30643E007F4
:10438100000043EB7F061218B9900D6F7405F080A1
:10439100597F0612290D900D6F7406F0804C7F062F
:1043A100124954900D6F7407F0803F7F06123D7CD7
:1043B100900D6F7408F080327F071218B9900D6F5D
:1043C1007409F080257F0712290D900D6F740AF092
:1043D10080187F07124954900D6F740BF0800B7F8A
:1043E10007123D7C900D6F740CF0D282C295900D36
:1043F1006FE0FF900D6EE0FD123FD3D295C2822295
:10440100900D6EEFF0121884442500443201443FB0
:1044110002444C034459044466054473064480072E
:104421000000448B7F081218B9900D6F740DF08055
:10443100597F0812290D900D6F7412F0804C7F087E
:10444100124954900D6F740FF0803F7F08123D7C2C
:10445100900D6F7410F080327F091218B9900D6FB2
:104461007411F080257F0912290D900D6F740EF0E3
:1044710080187F09124954900D6F7413F0800B7FDF
:1044810009123D7C900D6F7414F0D282C296900D8A
:104491006FE0FF900D6EE0FD123FD3D296C28222F3
:1052C700900D6EEFF024FA601704702B900D6F7439
:1052D7001DF0900D737403F07B277D2A7F1D8012CC
:1052E700900D6F741CF0900D737402F07B117D1F8D
:1052F7007F1C123822800A900D6EE0FFA3F0122661
:1053070092D282C294900D6FE0FF900D6EE0FD1275
:075317003FD3D294C28222B1
:10526F00900D6EEFF024FA601704702A900D6F7492
:10527F001BF0900D737401F07B287D2B7F1B801129
:10528F00900D6F741AF0E4900D73F07B127D207FF8
:10529F001A123822800C900D6EE02415FFA3F01225
:1052AF004708D282C297900D6FE0FF900D6EE0FD20
:0852BF00123FD3D297C28222F4
:0F6328009014697407F0D294D295D296D297222E
:105B4400C2AC123807EF12142E9014F11237B312AC
:105B5400380774019014EA6B7008E965827003EAEF
:0D5B6400658370069014F012380DD2AC224B
:10554900123816C003C002C001123807D082D083B6
:10555900D0E06B7008E965827003EA6583602B12FD
:1055690038161213C6FF1261389014F41237B312A9
:10557900381674019014EA6B7008E965827003EAC1
:0B558900658370069014F312380D22A9
:103A1E00900AF1E584F0ACA890133912182FE94AF8
:103A2E007003023B0653A87DE4F58453F87F90158E
:103A3E0030F0A3F0C2B3901427E0FFB40118901336
:103A4E0020E0C313FE7402A806088002C333D8FC1C
:103A5E00901530F08059EFB402169013F8E0FF7411
:103A6E0001A807088002C333D8FC901531F0803FBF
:103A7E00901427E0B40338901327E0C31314601595
:103A8E0014601A14601F14602424047022901531DF
:103A9E007410F0801A9015317420F0801290153148
:103AAE007440F0800A9015317480F08002D2B330E9
:103ABE001007901530E04440F0C2FAE4FF0FEFB467
:103ACE0032FB53F87FE59A20E7FB901530E0F59B2B
:103ADE00E4FF0FEFB432FB53F87FE59A20E7FB903B
:103AEE001531E0F59BE4FF0FEFB432FBD2FA900AEA
:093AFE00F1E0F584AF048FA82269
:031A060002415644
:10415600C0E0C0F0C083C082C0D075D000C000C02F
:1041660001C002C003C004C005C006C007C3901545
:104176002CE094F890152BE0942A50031237B39054
:104186001469E014F0E0C3940750067426F0125543
:1041960049901469E0FF131313541FFEEF54079060
:1041A6000D6DF0AF06EF24FE601814601F14602634
:1041B6002403702E900D6DE0FF640760251252C730
:1041C6008020900D6DE0FF1243618016900D6DE02A
:1041D600FF124401800C900D6DE0FF64076003122E
:1041E600526F758AFF758CFFD007D006D005D004B4
:1041F600D003D002D001D000D0D0D082D083D0F06E
:03420600D0E032D3
:1063090075F002EF90058012181AECF0A3EDF02257
:105AE8009015D0E0FEA3E0FF9015CCE0FCA3E0FD0C
:105AF800B50719ECB506159015D5E0FEA3E0FFED46
:0E5B0800B50709ECB5060520C502D322C3225D
:0A63EA00AE077F8B1237BA025B4446
:0A63F400AE077F821237BA025B4445
:0A63FE00AE077F831237BA025B443A
:104D6E00E4FE1237255012EE12370AE0F46007EE19
:104D7E00123734E004F00E80E99014FBE0FE123797
:104D8E000AEFF0123732E4F0FE1237255012EE120F
:104D9E00370AE0B4FF079014FBEEF0803B0E80E97B
:104DAE00E49014FBF09014ECE0FD7E0112372550D8
:104DBE0027EEFB3395E0FA74EC2BF58274143AF57A
:104DCE0083E0FCD3ED6480F8EC6480984007AD047A
:0C4DDE009014FBEEF00E80D41263F4225F
:10409700900ADBEFF0E4FF90128CE0D36480F8EF36
:1040A700648098506B123709E0FE900ADBE0FDEE62
:1040B7006D705912370974FFF012373874FFF0909A
:1040C7000ADC747FF0E4FE123725501CEE6F601592
:1040D700123732E0FD900ADCE0C36480F8ED6480BB
:1040E700985002EDF00E80DFE4FE1237255021EEE6
:1040F7006F6016123732C083C082E0FD900ADCE0A1
:10410700FCC3ED9CD082D083F00E80DE0F02409E70
:10411700E49014FBF0FF90128CE0FED36480F8EF7C
:104127006480985010123709E0F4601A9014FBE08D
:1041370004F00F80E1EE14FF9014FBE0FED3EF12C2
:0F414700372A4002EFF0900ADBE0FF1263FE22FE
:106138007584014398028F99E59870047F01800265
:0A6148007F00EF20E1F2E4F584226D
:1061CD00E4F5844398028F99E59870047F0180026D
:0761DD007F00EF20E1F22238
:105B7100E4FEC3EF12372A5023E4FDC3EF6480F83B
:105B8100ED6480985013E4FCC3EF6480F8EC64800A
:0D5B91009850030C80F20D80E20E80D622A9
:1062E700AE07ED60047F8F80027F8E1237BA025BA4
:0162F7004462
:100C9A00E490128CF0FBFAF990133912184F75FF91
:100CAA00DE75FFADE4F5E6F5E71261841262101213
:100CBA005888126328125EB31262F8E4F58475D478
:100CCA008475D48475D10375D340D281125C76D2EF
:100CDA00AFD2FFE4900AD1F090152A745AF0E4904A
:100CEA0014FBF0900AD1F090128CE0FF3395E0FEED
:100CFA00900AD1E0D39FEE6480F8748098501FE088
:100D0A00FF24F7F582E43414F58374FFF074EC2FB2
:100D1A00F582E43414F58374FF12375780C9E4125C
:100D2A0013BB124F50125EF6126408123A1E7F3934
:100D3A001261CDC20F1262C3EF640160030210E1B7
:100D4A0012604FEF64B060030210E1900AD8F0908D
:100D5A000AD1F01237C2942D501074FD2FF582E497
:100D6A003414F583E412375780E9E4900AD1F0127B
:100D7A0037C2941B501AE0FE2400123762E0FD7459
:100D8A00DE2E12378CEDF012375FE412375780DF10
:100D9A00C2001262C3EF60FA12604F900AD2EFF0FB
:100DAA005480FFE4FCFDFEEF7003020F1FE0FF64B6
:100DBA00C07003020F1FEF64B07003020F1F900A86
:100DCA00D8E004F0900AD2E0547FFF900AD4F0747D
:100DDA0019D39F500DE0FF94265007EF24F2A3F099
:100DEA00802A900AD4E0FFE4D39F500AEF94185067
:100DFA0005A3EFF08016EFB42908900AD57419F00C
:100E0A00800AEFB42C06900AD5741AF0900AD5E03D
:100E1A00FFC3941B502912375F7401F090152DEF10
:100E2A00F09014FCE0FF900AD5E06F600A90142756
:100E3A00E0B406031235E3900AD5E09014FCF0E41E
:100E4A00900AD6F0A3F01262C3EF60FA12604F90D4
:100E5A000AD3EFF01262C3EF60FA12604FAD079047
:100E6A000AD3E0FF900AD6E0F0A3E04FF0900AD64A
:100E7A00E0FEA3E07806C333CE33CED8F9F0EE9085
:100E8A000AD6F0AF05E0F0A3E04FF0900AD4E0757F
:100E9A00F00290058012181AE0FEA3E04E702F901F
:100EAA000AD1F01237C29405500C900AD4E090008F
:100EBA00F812374380EDE4900AD1F01237C2940455
:100ECA00500C900AD4E09001E112374380ED900A69
:100EDA00D4E0FF900AD6E0FCA3E0FD126309900A71
:100EEA00D4E0FF24FDF582E43414F5837401F09014
:100EFA0014F6EFF0C39419400CE0FFD39426500582
:100F0A00EF24F280049014F6E09014EBF020000530
:100F1A00125A88D200900AD2E064C06003020D9C83
:100F2A009013F7E0601E901427E0B402081251589B
:100F3A00301202C212901427E0B406081256273063
:100F4A001402C214E4900AD1F01237C2941B40036F
:100F5A000210E174DE2F12378CE0600302109590C4
:100F6A000AD1E02400123762E0640160030210959E
:100F7A00900AD9F0A3F0900AD9E0FEA3E0FFC39447
:100F8A0004EE64809480504590109875F07DEF12BD
:100F9A00181AEE75F07DA42583F583C083C082906C
:100FAA000AD1E0FFD082D08375F00512181AE054F6
:100FBA000F6012900AD9E0FCA3E024DAF5827405E6
:100FCA003CF583EFF0900AD91237B380A99013F752
:100FDA00E07008900AD1E0FF124D6E900AD1E0FF4E
:100FEA0012376E7414F0A3E4F0EF25E02496F5822C
:100FFA00E43400F583C083C082E04410FFA3E0D04C
:10100A0082D083CFF0A3EFF09013F7E070030210C1
:10101A00DBD212D214901427E0FF6402703F9013BF
:10102A003612182F900AD1E0FE75F005A4F58285D4
:10103A00F0831213DF540F70047D0180027D00EDEE
:10104A00540FFD90133612182F75F005EEA429F9E6
:10105A00EA35F0FA1213C654F04D12142EEF640654
:10106A007020900AD1E0FF244F1237CCE070047E42
:10107A000180027E001237C9EEF01237C9E0FD1274
:10108A0062E7121A1B1264080210DB123785E0B4F9
:10109A00010B12375FE070051240978034123785D2
:1010AA00E06401702C12375FE06401702412376A21
:1010BA00E0FCA3E0D39400EC9402400EEF12376EEA
:1010CA0074FE75F0001214FF800712376AE4F0A369
:1010DA00F0123758020F531262D5EF64016003020F
:1010EA0011C812606E900AD9EFF030E738E0901418
:1010FA00EAF0246824FC501D24E1601324D2600322
:10110A000211C81237FC90132412381C0211C8129B
:10111A0062B10211C89014EAE02468901468F0548D
:10112A0003F00211C89014EAE012188411B68C1167
:10113A00C08D115890116092117093119A9411A454
:10114A009511AC9611809711909D000011C8121349
:10115A00AF7492F08068900AD9E0FF12641190147B
:10116A00EA7493F08058900AD9E0FF12566F9014EF
:10117A00EA74F0F08048900AD9E0FF12638D901467
:10118A00EA749DF08038900AD9E0FF125E05802E3D
:10119A00900AD9E0FF12633780241213AF7496F0D5
:1011AA00801C900AD9E0FF12639A8012900AD9E053
:1011BA00FF1263468008900AD9E0FF126355126055
:1011CA00C8EF7003021295125A1F900AD9EFF01253
:1011DA001884124401123F02125704120B0512041A
:1011EA000612190712120812270912200A12350BC1
:1011FA00122E0C124C0D0000128612371A7FFF8035
:10120A002F12371A7F01802812371A7FFE80211287
:10121A00371A7F02801A12371A7FFD801312371A83
:10122A007F03800C12371A7FFC800512371A7F045D
:10123A001218AE8013121A21800E90135A12381CFB
:10124A00800690135712381C123A1E802F30111242
:10125A00B2103010047F8980027F8A900AD4EFF09E
:10126A00800FE490101EF01261B5C2107FBA125BB3
:10127A0044123A1E900AD4E0FF1261381260C8EF95
:10128A0060030211D11237FC126408125AB8EF70C7
:10129A0003020D3D301021901601E014600F047016
:1012AA0017901602E01213BB126408800B90160204
:1012BA00E090101EF01261B5901601E0FFB40B0227
:1012CA00D211EF6431701E12377A7019125AE8502F
:1012DA00FB121392A3E0900ADEF0123BE7125AE8DF
:1012EA0050FB1213A6901601E06432701812377A76
:1012FA007013125AE850FB121392123E44125AE823
:10130A0050FB1213A6901601E0642D702A12377A48
:10131A007025125AE850FB90152AE0FF12624F120C
:10132A005AE850FB1237E51245D7125AE850FB909B
:10133A00152AE0FF12623A901601E0642E702A1212
:10134A00377A7025125AE850FB90152AE0FF12628C
:10135A004F125AE850FB1237E51247A0125AE850CA
:10136A00FB90152AE0FF12623A901601E0B41405C8
:10137A00D210123A1E901601E064156003020D3D68
:10138A00C210123A1E020D3D90152AE0FF12624F5A
:10139A00901603E0FFA3E0FDA3E0FB2290152AE0EC
:1013AA00FF12623A22900AD9E0FF1264699014EAA5
:0C13BA002290101EF0125C4C1263E02226
:102DC1004C00500049002000540043560050756CDF
:102DD1007320313A2573257320323A257325730008
:102DE100333A2573257320343A2573257320353AF8
:102DF100257325730043562031303A2573257320FE
:102E010031313A257325730031323A257325732008
:102E110031333A2573257331343A257325730043D1
:102E21006F6E747261737420256420006F66660092
:102E3100363700363738003637383900506F6C79FD
:102E410070686F6E792025732000526973696E670F
:102E51000046616C6C696E6700547269616E676CE3
:102E6100650052616E646F6D0053706972616C0030
:102E71002030002E35002031002032002033002088
:102E81003400203600203800313000313500323036
:102E910000323500333000417270656767696F2019
:102EA10025733A202573004B59006B790043563A3C
:102EB100252D33642054723A25642025632564004E
:102EC100506174726E3A2025730046616465206911
:102ED1006E3A2573206F7574257300526164696FB2
:102EE1003A25642025733A25732025732000435623
:102EF100313A252D3364204356323A25642000436C
:102F010056313A252D3364204356323A2573200039
:102F11006C6F6300FF2DC102FF2DC303FF2DC5049C
:102F2100FF2DC700FF2DC906FF2DCB05FF2DC102C7
:102F3100000600070008000900050009000D001146
:102F41000007FF1A010008FF1A12000CFF647B0042
:102F51000DFF644D0102FF64800103FF645401070A
:102F6100FF64850108FF645B010CFF648A010DFFAA
:102F710064620006FF34B80008FF619D000BFF5A30
:102F810055000DFF48380105FF54FD010DFF4B6E43
:102F91000006FF648F0007FF642A000CFF649400A1
:102FA1000DFF64310103FF64990104FF64380109D5
:102FB100FF649E010AFF643F010EFF64A3010FFF3E
:102FC10064460009FF61520109FF6152000AFF5B7B
:102FD1009E010AFF5B9E000AFF619D000DFF49DF14
:102FE1000104FF4C70010AFF5ED5010DFF3CB400E6
:0E2FF10007FF5CC90108FF5F76010FFF5F95C7
:10338300411320004113210041132700411328005A
:103393004113290041132A0041132D004313360022
:1033A300000041142202411427014113F80059136C
:1033B300C56162636465666768696A6B6C6D6E6F2D
:1033C300707172737475767778795913DE4142435D
:1033D3004445464748494A4B4C4D4E4F5051525332
:1033E3005455565758594113F70043143D0113C51B
:1033F30041142C0041141F0041143B0241133E00B1
:1034030041142D0041143C0041143A324114680028
:103413004812D300FA00FA00FA00FA411428000C0B
:1034230009FF2E2DFF2E31FF2E34FF2E384F14406F
:10343300FF2E4BFF2E52FF2E5AFF2E63FF2E6A6084
:103443002712F9FF2E71FF2E74FF2E77FF2E7AFFBE
:103453002E7DFF2E80FF2E83FF2E86FF2E89FF2ECB
:103463008CFF2E8FFF2E92FF2E950108010215006F
:013473000157
:1020D000EDFF3395E0FE75F003EF12181AEE75F080
:1020E00003A42583F583227A14790E900AE47B01F8
:1020F00012184F7A1379FB2224C590143D7B01F905
:10210000E43413FA02184F9012DB75F003ED121845
:102110001AEC22EFF0A2AFE433A3F0125E29C2AFB3
:102120009014287401F0EF75F005A4FF90133602A7
:10213000182F24C5F9E43413FA12184F0213C67B82
:10214000FF900AE402184F901468E025E024D3F5CC
:1021500082E43412F583229013F8E075F07DA42414
:1021600098F9741035F0FA7B0190133602184F126B
:10217000182F121864900AE712184F7B012290144E
:102180003D12182F9013C5C3E99582EA9583222446
:10219000DEF9E4341390143DFA7B0102184F9014D9
:1021A0003D12182F0213C69013F8E075F002A4FF39
:1021B000AEF02431F9742F3EFA7BFF9013401218D1
:1021C0004F74392FF9742F3EFA90142922FD901480
:1021D0002912182F12152BAEF07802227BFF9013D4
:1021E0005702184F7B0190133902184F900ADDE017
:1021F000FFA3E0CF900AE7F0A3EFF02212182F120E
:102200001864900AED02184F900AEA12182F74020F
:1022100012142E7BFF7A2F791522E024C5F9E434BD
:1022200013FA22900AE512182F90000322FF901350
:1022300022E04EFEA3E04FFFEE901322F0A3EFF05A
:1022400022744F2FF582E43414F583229013240274
:10225000184F90135A02184FEDFF3395E0FE227588
:10226000F005EFA429F9EA35F0FA0213C690143DFF
:1022700002182F740312142E7BFF7A2F791922EF84
:10228000F090134012182F02152BE075F003A424D0
:10229000F9F582E43412F58302182F7B01E0FD90FA
:1022A0000AE822901427F07BFF22D3EF6480948009
:1022B00022900AEA02184F12182F121864900AF39B
:1022C00012184F7B012275F003A4242EF582E4340A
:1022D00014F5832275F005A4245FF582E43413F528
:1022E000832275F005A4245DF582E43413F583227E
:1022F00075F005A4245EF582E43413F58322E0FE34
:10230000A3E09012DB75F00322C390152CE094102B
:1023100090152BE094272290132412182FEB8A8318
:1023200089827BFF22900AE3E4F0A3227BFF7A2FCD
:10233000791D22121556FFAEF0D39400EE94FE22C2
:102340007B017A14790E22E025E02492F582E434B0
:1023500012F58322EFF0D36480948022900AE37414
:10236000FFF0A32290128CE0C3648022E49013F764
:10237000F07F03227B01E0FD900AE8740DF022E07B
:1023800024FF92AFE4901428F022900AF612184F1E
:102390007A14790E22E025E02406A3F02290142777
:1023A000F07BFF222423F58274103EF5832212185D
:1023B0002F74019013D66B2212182F74019013D72B
:0C23C0006B222427F58274103EF5832266
:104F50007F1990144FE4F0A3DFFC7B017A1079985D
:104F60001221697BFF7A2F793190134012184F7A02
:104F70002F793990142912184F12219E901343F063
:104F8000E4A3F09013C1F0FF122213EF1222C61215
:104F9000184F0FEFB404F1E49013FAF090140DF0F1
:104FA000901421F0901424F0901426F090132CF01B
:104FB00090132FF0901331F0901333F0901335F0DD
:014FC00022CE
:061A0900E490133FF022FF
:10509900900AE1EEF0A3EFF0AF051DEF6053900A1F
:1050A900E1E0FEA3E0F5828E83A3A31218589013C2
:1050B9003FE0FF1222D412184F900AE1E0FAA3E070
:1050C900FBF5828A83E493FEEF1222E2EEF08B82F3
:1050D9008A83740193FF90133FE01222F0EFF0905E
:1050E900133FE004F0900AE1E475F0051214FF8023
:0250F900A722EC
:105D44009013391221A1FE1222E2E0FFEE1222F09A
:105D5400E0FD1263B29013391221A11222D4121859
:075D64002F90135402184FA9
:101A210090133912182F740112140C9013391221CA
:0E1A3100A1FF90133FE0B50704E412142E222B
:105CA000D3ED6480948040047401800274FF121468
:105CB0000C1213C6FFB4FF03E4800A900AE8E0FE6A
:095CC000B50705EE1412142E22A2
:106152007B017A147922AD07900AE87408F0125C88
:09616200A0901422E0FF0263D5B5
:105B9E007B017A12798CAD07900AE87404F0125CDE
:105BAE00A0E49013F8F0E075F07DA42498F9741039
:0C5BBE0035F0FA1221691221A702184FDD
:1049DF00900AE3EFF0E49013F7F0125CF212217EED
:1049EF00401512226DD39013DD1221885009122227
:1049FF006DC3E994C5800712226DC3E994DE900A56
:104A0F00E4F0900AE3E0FED3648094804019A3E0C1
:104A1F00FF12218FE4D39F5026EFC3941950201219
:104A2F0022417401F08018900AE4E0FF1220F8E4AC
:104A3F00D39F500BEFC394195005122241E4F0900D
:104A4F000AE4E0FFD3EE6480948040047D0180028D
:084A5F007D001262E7021A1B40
:104C70009014EBE0FEE4D39E5074EEC39419506E92
:104C8000EF1218844CA0014CB0024CC0034CD0046D
:104C90004CD8FC4CC8FD4CB8FE4CA8FF00004CDEC4
:104CA000900AE374A0F08036900AE374A4F0802E9A
:104CB000900AE374A1F08026900AE374A5F0801EA8
:104CC000900AE374A2F08016900AE374A6F0800EB6
:104CD000900AE374A3F08006900AE374A7F0900AA8
:0F4CE000E3E0FF125B449014EBE0FF125B442211
:105CC900900AE3EFF0BF01047FB48009900AE3E092
:105CD900B4FF057FB5125B447A13793E900AE3124B
:095CE900229B7405F0125CA0225C
:105ED500900AE312235440047FB280027FB3125B21
:105EE500447A147968900AE312229B7404F0025CE8
:015EF500A00C
:103CB400EF1218843CD4013CED023D05033D1D0484
:103CC4003D29FC3D11FD3CF9FE3CDFFF00003D3386
:103CD40012232504F0A374A8F0805474FF900AE31F
:103CE400F0A3F0A374ACF080461223257410F0A363
:103CF40074A9F0803A12235C74F0F0A374ADF080E0
:103D04002E1223257440F0A374AAF0802212235C9F
:103D140074C0F0A374AEF08016122325747FF0A350
:103D240074ABF0800A12235C7481F0A374AFF0903A
:103D34000AE5E0FF125B44900AE3E0FEA3E0FF9093
:103D44001468E0FD12214BEE8FF01214FFED1221E6
:103D54004BE0FEA3E0D394F4EE9401400CED122169
:103D64004B7401F0A374F4F022C3EE94005008EDF8
:083D740012214BE4F0A3F02240
:105F7600900AE312235440047FB680027FB7125B77
:0F5F8600447A14792D900AE3122374125CA0223E
:105F9500900AE312235440047FB880027FB9125B54
:0F5FA500447A14793C900AE3122374125CA02210
:0964080090132412182F0218AAA7
:105EF6009014277401F07A5E79911221DC7A4D793B
:105F0600EA12224C7A5F79161222527F010263EA64
:105F16009014277402F07A5E79F61221DC7A3179D0
:105F2600AB12224C7A5F79B41222527F020263EAE4
:105FB40074031222A37A5F79161221DE7A4879C714
:0F5FC40012224C7A5F79D31222527F030263EAD2
:105FD30074041222A37A5F79B41221DE7A5579DF31
:0F5FE30012224C7A5F79F21222527F040263EA93
:105FF200740512239D7A5F79D31221DE7A57793D97
:0F60020012224C7A6079111222527F050263EA52
:10601100740612239D7A5F79F21221DE7A3579E3D3
:0F60210012224C7A5E79911222527F060263EAB4
:105E91009014277407F07BFF7A6079111221DE7A62
:105EA1004E79DC12224C7A5E79F61222527F070279
:025EB10063EAA2
:1056F900AD07ED3395E0FEEF7802C333CE33CED854
:10570900F9244FF974103E900AE5122198AF05EF7C
:105719003395E0FE9012A61220D612182F900AE8AF
:1057290012184F900AE51221A1B40205740312144C
:045739002E021A1B07
:10584B001222AA7BFF40067A2F792580047A2F79C2
:10585B00219013451220D012184F12225890134545
:10586B001220D61222261213DFFCEF7802C333CE9E
:0D587B0033CED8F91223A4ECF0121A1B2230
:051A0100E4FD02584B5A
:05647B007D0102584BF9
:056480007D0202584BF3
:056485007D0302584BED
:05648A007D0402584BE7
:104AED00900AEA12184F1222AA4026900AEA1221C1
:104AFD00A124FE600A1460091460062404705F800E
:104B0D0024900AEA12182F740412142E12232C80EA
:104B1D0047900AEA1221A124FE600F14601114605F
:104B2D002E24047039122273802E122208802990AF
:104B3D000AF0E075F003A424CCF582E43412F58379
:104B4D001221A1D3648094EB4014122208800990A5
:104B5D000AEA12182F122273900AED12184F021A38
:014B6D001B2C
:10546400AC07122258EF7802C333CE33CED8F924D6
:105474004FF974103EFA7B01900AE312184F12227E
:10548400589012A61220D612182F900AE612184F1E
:10549400AF04900AE612182F900AED12184F900AE2
:0D54A400F0EDF0900AE312182F124AED22ED
:05648F007D0A025464C7
:056494007D0B025464C1
:056499007D0C025464BB
:05649E007D0D025464B5
:0564A3007D0E025464AF
:103F0C001222AA40431221071220DEA3E475F0010D
:103F1C001214FF30017C1221071220DE1223AE7026
:103F2C0008E965827003EA65836015122107122087
:103F3C00DE1223B87008E965827003EA658370525B
:103F4C007B017A1379D880411221071220DEA374E9
:103F5C00FFF5F01214FF3001391221071220DE1286
:103F6C0023AE7008E965827003EA6583601512213F
:103F7C00071220DE1223B87008E965827003EA6527
:103F8C0083700F7B017A1379D51221071220DE1270
:103F9C00184F1221071220DE12182FD39013DD12A6
:103FAC00218840087B017A1379DD801112210712D8
:103FBC0020DE122181500F7B017A1379C512210763
:073FCC001220DE12184F2243
:10593C00900AE3ECF0A3EDF0C201123F0C900AE3E5
:10594C001222FE1220DA12182FC3E994C5FD900A18
:10595C00E3A3E07802C333CE33CED8F92422F58208
:0A596C0074103EF583EDF0021A1BE3
:1050FB00900AE3ECF0A3EDF0D201123F0C900AE31F
:10510B001222FE1220DA12182FC3E994C5FD900A61
:10511B00E3E0FAA3E0FB7802C333CE33CED8F92415
:10512B0062F58274103EF583EDF0122302EB121838
:10513B001AEA1220DE1221A1C3648094EC500B906A
:0D514B000AE3A3E02405FF1256F9021A1B27
:07642A007D057C000250FB20
:076431007D067C000250FB18
:076438007D077C000250FB10
:07643F007D087C000250FB08
:076446007D097C000250FB00
:061A1200E4FDFC02593C5A
:07644D007D017C0002593CB7
:076454007D027C0002593CAF
:07645B007D037C0002593CA7
:076462007D047C0002593C9F
:1034B8001222AA500302354E12212C740190109842
:1034C8006B7008E965827003EA6583702090128C3E
:1034D800E0146012146011146010240370629013D9
:1034E800F87401F0805A801A8035E4804F12212C3C
:1034F80074019011156B7008E965827003EA6583A1
:1035080070089013F87402F0803612212C74019020
:1035180011926B7008E965827003EA658370089000
:1035280013F87403F0801912212C740190120F6B98
:103538007008E965827003EA658370049013F8F0F7
:103548001221570235D912212C74019010986B70F2
:1035580008E965827003EA6583700F122364948317
:1035680050439013F87403F0806712212C74019073
:1035780011156B7008E965827003EA658370028033
:103588004C12212C74019011926B7008E9658270BD
:1035980003EA65837012122364948150089013F82B
:1035A8007401F0802CE4802512212C740190120FF4
:1035B8006B7008E965827003EA65837014122364EE
:1035C800948250089013F87402F08005E49013F880
:0B35D800F01221571221A712184F22F9
:10619D001222AA40079013F77401F02212236C12F9
:0861AD005B717F391261CD2204
:105E290012217E401512226DD39013DD1221885064
:105E39000912226DC3E994C5FF2212226DC3E994A8
:035E4900DEFF2257
:105A5500AE07125E29D3EE64809480401274DE2F67
:105A650012219112212C12225F54F04401800E74F0
:105A7500C52F1220FA12212C12225F54F012142E77
:035A8500021A1BE7
:10483800900AE312227F24FAFFE5F034FFFE900A83
:10484800E3E0D36480948090142E75F003EF400A5F
:104858001220DAA3E475F00480091220DAA374FFA9
:1048680075F0FC1214FF90142E1220D612182FD3B4
:10487800902F1D122188400C12232C90142E1220E8
:10488800D612184F90142E1220D612182F902F15CA
:10489800122187500C12221390142E1220D61218AF
:1048A8004F90142E1220D61222261213DF1221CD79
:0F48B800C333CE33CED8F91223C2EDF0021A1B50
:1054B100EF12188454D10154DB0254E50354EF0474
:1054C10054F4FC54EAFD54E0FE54D6FF000054F9B4
:1054D1007E007F01227EFF7FFF227E007F10227EE1
:1054E100FF7FF0227E007F40227EFF7FC0227E0070
:0C54F1007FFF227EFF7F0122E4FEFF22ED
:1054FD00900AE3122113E92FF9EA35F0FA900AE345
:10550D00E0FF1254B1900001EE8FF012158E900055
:10551D00011223334008900001E4F5F08011C3EF30
:10552D0094C6EE9403400B900001740375F0C612FF
:0C553D0015DB121A1B900AE412237F22D7
:104B6E00900AE3122113E92FF9EA35F0FA900AE5DB
:104B7E0012184F1221CEC333CE33CED8F9242CF9CE
:104B8E0074103EFA7B01900AE812184F900AE3E087
:104B9E00FF1254B1122223EE8FF012158E900003E5
:104BAE001223334013122223E4F5F01215DB900A80
:104BBE00E81222267402801CC3EF94C6EE940340C2
:104BCE000B122223740375F0C61215DB900AE8123D
:104BDE0022267405121440121A1B900AE412237F27
:014BEE0022A4
:10467000901076E024C59012EA1220FD1213C69025
:10468000132BF090107AE024C59012ED1220FF1247
:1046900013C690132EF090107EE09012F01221328B
:1046A000901330F0901082E09012F31221329013A8
:1046B00032F090108612221A9012F61221399013BD
:1046C00034F0E4FD122258EF7802C333CE33CED853
:1046D000F92477F58274103EF583E0601024FD60C4
:1046E0000C14600E24027019122213800812227812
:1046F000800312232C1222589012C41220D61218B2
:084700004F0DED640570BD22B0
:104DEA00124A677A2D79CE12213F90134512216F0C
:104DFA007A1379F91222B19013481221FC7A1479A4
:104E0A000C900AF01220EE121AA77A2D79E11221DB
:104E1A003F90134B12216F7A1479201222B190130A
:104E2A004E1221FC7B017A147923900AF012184F52
:104E3A009013511222B77A14792512238A121AA7CB
:104E4A001220E7125976121A097E2F7F417D0A1223
:0C4E5A0050997A1379201221E4025D4483
:1048C70012236C125B717F391261CD1246707BFF28
:1048D7007A2D79F61221419012C412216F7A137939
:1048E7002B1222B19012C71221FC7B017A13792E69
:1048F700900AF01220F0121AA77BFF7A2E7909127C
:1049070021419012CA12216F7A1379301222B19085
:1049170012CD1221FC7B017A137932900AF012181A
:104927004F9012D01222B77A13793412238A121AAF
:10493700A71220E7125976121A097E2F7F917D0A56
:0D4947001250997A1379271221E4025D4481
:1055DF007BFF7A2E7920122141901422E0FFE412F2
:1055EF0021F47B017A1379FB121AA77BFF7A2D79AD
:1055FF00C7122141122340121AA71220E71259761F
:10560F00121A097E2F7FC37D011250997B017A13E5
:08561F0079281221E6025D4426
:10573D007BFF7A2E793D12214190128CE075F0039A
:10574D00A42409F81218261221757A1379FB121A5E
:10575D00A7E490140EF01220E7125976121A097E62
:10576D002F7FCD7D011250997B017A13792912215A
:04577D00E6025D449F
:1035E3009013F7E0600D7F03125B717F381261CD9A
:1035F30012562790132AE0B40205E49013F7F090D3
:1036030014EBE0FF6411600BEF64126006EFC394E8
:10361300194008901290E09014EBF09014EBE0FF47
:10362300E4D39F40030236DFEFC39419400302360D
:10363300DF122241E09014EB6009E024DEF9E43468
:10364300138007E024C5F9E4341312219512219E57
:10365300901343F07BFF7A2E79981221419013F750
:10366300E060067A2E79A880067BFF7A2E79AB126A
:1036730021757A137943900AEA1220F0121AA712DD
:103683002147E0FEA3E02406FFEE34FFFE1263BEF3
:10369300900AECEEF0A3EFF07BFF7A2E79AE1221C5
:1036A300419014EB1223471221EF901468E0FF249A
:1036B30001FCE433900AE9F0A3CCF0EF12214BE0D4
:1036C300FEA3E0C394FAEE940050047F2D80027FA2
:1036D30020900AEBEFF0122340121AA7122309409D
:1036E3000D1220E7125976E490152BF0A3F0121A6D
:1036F300097E2F7FD77D051250997B017A13792A92
:063703001221E6025D4404
:104EDC0012236C125B717F391261CD7BFF7A2E79B4
:104EEC00C112214190133EE075F003A42440F582D9
:104EFC00E43414F58312182F1221757A1379FB12EE
:104F0C001AA77BFF7A2E79CB12214190142D1222F5
:104F1C008A900AE712184F90143C12228A1222B17E
:104F2C00122340121AA71220E7125976121A097E80
:104F3C002F7FF07D031250997B017A13792D12216A
:044F4C00E6025D44D8
:104A670090102212221A7B019012DB122139901327
:104A7700F9F090102612221A9012DE1221399014A2
:104A87000CF090102A12221A9012E1122139901478
:104A970020F090102E12221A9012E412213990144D
:104AA70023F090103212221A9012E7122139901433
:104AB70025F0E4FD122258EF7802C333CE33CED867
:104AC700F91223A4E07BFFB406067A2F7925800428
:104AD7007A2F79211222589013451220D612184F97
:064AE7000DEDB405CF2225
:105A88001223177A3179ABF4700A74AB658270040B
:105A98007431658360161223177A3579E3F4700A36
:105AA80074E3658270047435658370031264082298
:10562700E4900ADBF0900ADBE0FFC36480949950B2
:1056370036EF3395E0FE744F2FF58274143EF583F1
:10564700E0900ADB6009E025E02407A3F08003125D
:1056570023957F03125B71900ADCE0FF1261CD9006
:085667000ADBE004F080BE2222
:10515800E4900AE1F0900AE1E0FFC364809499507A
:105168004B9013F8E075F07D90109812181AEF33F1
:1051780095E0FE75F005EF12181AEE75F005A425F6
:1051880083F583E0540F900AE16009E025E02407E5
:10519800A3F080031223957F03125B71900AE2E06B
:0D51A800FF1261CD900AE1E004F080A92221
:105CF200E4900AE5F0900AE5E0FFC394195019EF29
:105D02001223967F0A125B71900AE6E0FF1261CDC0
:095D1200900AE5E004F080DD22B6
:1031AB009013F7E0600D7F03125B717F381261CDD6
:1031BB001251589014EBE0FF125BCA500890129119
:1031CB00E09014EBF09014EBE0FF642C6004EFB490
:1031DB002908901291E09014EBF09014EBE0FF9023
:1031EB001291F012212C75F005EFA4F58285F08376
:1031FB001213DF540F9014EB600AE012218FC3E916
:10320B0094DE8008E01220F8C3E994C5900ADBF045
:10321B00900ADBE0122127E92F122265C4540F908C
:10322B000ADCF0900001121556FF900ADDE5F0F074
:10323B00A3EFF0900003121556FF900ADFE5F0F0B4
:10324B00A312227F24FA1221CDC333CE33CED8F969
:10325B001223C2E024FE600A14600C14600E2404D6
:10326B0070161222138008122278800312232C90DE
:10327B00142E1220D012184F12219E901343F07B64
:10328B00FF7A2E79DC122141122281FF900AE7E5A9
:10329B00F0F0A3EFF09013F7E07BFF60067A2E7946
:1032AB00A880047A2E79AB900AE912184F7B017A29
:1032BB00137943900AEC12184FED1222C612182FF5
:1032CB00121864900AEF12184F7B017A1379FB12D4
:1032DB001AA71221CEC333CE33CED8F9242FF582C1
:1032EB0074103EF583E07BFFB4051B7A2E79EF1249
:1032FB0021411221EC900ADFE0FFA3E0900AE9CF15
:10330B00F0A3EFF080127A2F79001221411221ECF9
:10331B007A2F7911A312184F122340121AA71223D6
:10332B0009400D1220E7125976E490152BF0A3F00B
:10333B00121A097E2F7F737D061250997B017A1327
:08334B0079211221E6025D4424
:0664690090133CEFF0224D
:09641100EF543FFFE4122239228E
:10566F007E00EF7806C333CE33CED8F912222DD376
:10567F0094C6EE9403400A9013227403F0A374C6E9
:10568F00F090133CE0FFE4D39F5019EFC3941950EF
:10569F0013901322E0FEA3E0FF90133C122347EE7A
:0556AF00F0A3EFF02262
:0C639A0090133CE0244F122244EFF0224C
:0D638D00EF543FFF901322E4F0A3EFF02245
:105E05007E00EF7806C333CE33CED8F912222DD3D8
:105E150094F4EE940140047E017FF4122147EEF0E4
:045E2500A3EFF022D5
:0F63370090133EEFF0E0C3940540037404F0228E
:0F63460090142DEFF0E0C3940D4003740CF0227F
:0F63550090143CEFF0E0C3940D4003740CF02261
:073474004405FC05090D11E0
:101DA7003EF583ECF0A3EDF0C3ED9BFDEC9AFCE967
:101DB700FF3395E0FEEF25E0FFEE33FE22ED75F0F1
:101DC7002DA424F8F582E43400F583E5822EF5820C
:101DD700E43583F58322E025E0249CF582E434058D
:101DE700F583E0FCA3E0FDEF25E02480F582E434F1
:101DF70005F583E0FEA3E0229005F912184F900D38
:101E070070E0901020FF75F00402181AE09005F9B1
:101E170075F07DA42498F9741035F0FA7B01021847
:101E27004F3EF583ECF0A3EDF022901023EF75F011
:101E37000402181AE4121440900D70E025E02424DF
:101E4700F822E0FF75F005A4F58285F0831213DF11
:101E5700540F22EF75F005A4FF9005F902182F74AF
:101E6700FFF5F0121515FCD3E5F09400EC648094AF
:101E77008022900D71E090102375F00412181AE07B
:101E870022E4F0EF24FAA3F0E0FD24FCF582E43429
:101E970005F583E022EF90102075F00402181A90E0
:101EA7000001E92FF9EA35F0FA121556FFAEF022D4
:101EB7003EF583E0FCA3E0FD2274802FF5827405D4
:101EC7003E222DFFEE3CFEF0A3EFF07C007D0502E5
:101ED7001462E0FE75F02DA424E1F582E43401F5E7
:101EE70083E5822F22FF900D84E0FCA3E0FD22E032
:101EF70024F7F582E43414F583E022EF25E0242467
:101F0700F8760F0876FF22900D84EEF0A3EFF0220B
:101F1700900D84E025E0FF900D83E033FE74B92F28
:101F2700F582740422A804A905AA06AB07E0FEA35C
:101F3700E0FF22E025E02480F582E43405F583E024
:101F470022FFE4FCFD0217CCFF7B1FE4FCFDFAF93E
:101F5700F80216157B017A1079989005F902184F47
:101F6700E024DAF582E43405F58322E47F2C7E0150
:101F7700FDFC12178BC3021732900D7FE0FCA3E024
:101F8700FD22F583E4F0A3F0EF25E0229005FAE4C3
:101F970075F0051214FF900D71E004F02275F02D15
:101FA700A424EFF582E43401F583E5822F22E9D3F7
:101FB7006480F8740B64809822E0FEA3E0FFED25AF
:101FC700E02424F8A60608A60722900D81EEF0A3C8
:101FD700EFF022900D72EEF0A3EFF00D1214C990FE
:101FE7000D72EE2290128CE0D3648022E4F0ED753E
:101FF700F02DA422741B2FF582740622E4FCFD0247
:1020070017CC74932FF582740622EF25E02424F869
:10201700E6FC08E622AB07AA06A905A80402177F73
:10202700E0A3FFE0FCA3E0FD22900D73E0FF3395F2
:10203700E0FEEF2274962FF58274003E22F0AF0582
:10204700125594EF4E22E4F0A37405F022D39400C6
:10205700EE9400221216087805121759AD07AC0640
:1020670022900D7212182F8F827583002274002F11
:10207700F58274002274572FF582740622745A2F42
:10208700F58274002275F004EE12181A7405F02216
:1020970025E02424F876080876002225E02424F891
:1020A700E4F608F622E0FF740BD39F222470F58232
:1020B70074053EF583221217CC900D7402177F9F8B
:0920C700EE6480F8EC64809822BC
:10559400AD07EDB4010F121FEB94807E0040037F32
:1055A40001227F0022EDB4020F121FEB94817E00D2
:1055B40040037F01227F0022EDB4030F121FEB94FE
:1055C400827E0040037F01227F0022121FEB948021
:0B55D4007E0040047F0180027F002267
:105EB300E4FFEF25E02400F582E43400121F892477
:105EC300B9F582E43404F583E4F0A3F00FEFB42DC5
:025ED300E122CA
:105BCA00EF64116022EF6412601DEF641F6018EF2A
:105BDA0064206013EF6428600EEF642B6009EF64A1
:0C5BEA00276004EFB42A03D38001C3221B
:1060E5009014F6E0FF7419D39F500BEF94265006D9
:0C60F500C3EF940EFF229014F6E0FF228F
:10453D00E4FF121E317406F00FEFB405F5E4FF74BD
:10454D00FC2F121E93FE74DA2F121F6AE4F0EE9008
:10455D001027121EA07402F090102B12208C9010B8
:10456D002F12208C0FEFB404D6E4FF74002FF582C8
:10457D00E43406F583E4F074DE2FF582E43405F5BA
:10458D0083E4F00FEFB41BE3E4FFEF25E0241BF50C
:10459D0082E43406121F892457F582E43406F5832C
:1045AD007401F0A37490F0EF25E02493F582E434C8
:1045BD0006121F89245AF582E43400F5837401F044
:0A45CD00A3742CF00FEFB41EC122FE
:1060AB00122011D39400EC94004005EF1220A22291
:0D60BB00901020121E3412204D121F0222E0
:105E4C00121E9C121E665011121E9C121F8B1220C9
:105E5C00144C600EEF122097221220114C6003128A
:035E6C001F0222F0
:104CEF00AE07C20D125BCA5032121DC4E06029120A
:104CFF001DC4121FF32406F582E43401121DD012D5
:104D0F001FF3240EF582E43401121DD0121FF32479
:104D1F0011F582E434018037024D68740BD39E5035
:104D2F001CEE94185017121DC4E0600F121DC41210
:104D3F001FF32406F582E434018014801C121DC475
:104D4F00E06016ED75F02DA424F8F582E43400121E
:0F4D5F001DD0E4F0AF050260ABAF05125E4C2231
:10269200900D70EFF0C20AC20BC20CE075F02DA4CF
:1026A20024F8F9740035F0FA7B01900D7212184F7C
:1026B200900D70E0901022121E0CE0900D71F0123D
:1026C2001E31E0B4060D900D71E0FF900D70E0FD3B
:1026D200024CEF900D711220AC5014EF9418500F71
:1026E200EF64116004EFB41204D20C8002D20B30FA
:1026F2000B4D1220681213DF6015900D71E0F58208
:10270200758300121E3BE6FE08E64E7002D20A9066
:102712000D71E0240EFFE433FEA312182F8F828E78
:10272200831213DF70030228078F828E83121E3BEF
:10273200E6FE08E64E6003022807D20A02280720B6
:102742000C030227E9900D71E064117048A312187E
:102752002F9000111213DF701890001F1213DF70F8
:10276200109000271213DF700890002A1213DF6006
:1027720024900011E412144090001FE412144090BF
:102782000027E412144090002A121E3BE6FE08E6DF
:102792004E7002D20A900D71E064127068A3121892
:1027A2002F9000121213DF70189000201213DF70A6
:1027B200109000281213DF700890002B1213DF60B4
:1027C20044900012E4121440900020E4121440904D
:1027D2000028E412144090002B121E3BE6FE08E68D
:1027E2004E7022D20A801E900D7212182F900D7117
:1027F200E0FFF5827583001213DF6009122068E49E
:10280200121440D20A300A0D900D70121E081220C6
:102812004DEF022909900D70121E08121E66400328
:10282200022905121E9CE4F0A3F0300B28900D71D2
:10283200E0FF121F3BFCA3E0D39400EC9400505D38
:10284200EF25E0249CF582E43405121DF812205491
:10285200404D0228E1200C030228ED900D71E0FFAB
:102862006411703DD39005A3E094009005A2E0941A
:1028720000502A9005D5E094009005D4E0940050D1
:102882001C9005CFE094009005CEE09400500E908D
:1028920005BFE094009005BEE094004002804080B5
:1028A20044EF64127064D39005A5E094009005A4EF
:1028B200E09400502A9005D7E094009005D6E09469
:1028C20000501C9005D1E094009005D0E094005097
:1028D2000E9005C1E094009005C0E094004006907F
:1028E2000D70E08016900D70E08014900D71E01272
:1028F2001DEF122054900D70E04004122097221216
:0B29020020A222900D70E0121F0322A3
:1018B900C20AEF24FA900D72F0E0FF121E91900D0A
:1018C90070F0125594EF4E60747B017A107998127A
:1018D9001DFF121E66505F121E9CE4F0A3F0900DCE
:1018E90071F0900D71E0FFC39419503B121E601204
:1018F90013C6540F602C900D72121EF6FEF460226E
:10190900EF6E701E900D71A3121ED9121DD5E060E5
:101919000302198E900D71E0121DEF12205440023E
:10192900D20A121F9380BB900D70121E42300A0317
:101939000219EA0219F0900D70E00219C9900D72AE
:10194900E075F07DA42498F9741035F0FA7B011242
:101959001DFF121E6640030219F5121E9CE4F0A336
:10196900F0900D71F0900D71E0FFC3941950691258
:101979001E601213C6540F6059900D72121ED912AF
:101989001DD5E06012EE121EDB121DD5E4F0121E09
:101999000512204DEF8029900D71E0FFEE121FA472
:1019A900121DD5E0601EEFD3940A4018900D71A363
:1019B900E0121FA4121DD5E4F0121E0512204DEFEE
:1019C900121F0322900D71E0121DEF1220544002E4
:1019D900D20A121F9302196E900D70121E42300A1C
:1019E90006760808760022E4F608F622900D7012B1
:0819F9001E42760F0876FF2262
:1023CC00900D7EEFF0A3EDF0F912203425E0FBEE3A
:1023DC0033FA745F2BF58274043A121DF8900D9445
:1023EC00121F48747B2BF58274043A121DF8900D61
:1023FC0098121F48121FB54003022691900D7FE0E2
:10240C00FF648094984003022691125BCA50030229
:10241C002691900D7FE0F9FB3395E0FAEB25E0FF78
:10242C00EA33FE74052FF5827404121EB7745F2F05
:10243C00F5827404121E2874212FF5827404121E66
:10244C00B7747B2FF5827404121E2874AB2FF5829F
:10245C007403121EB774052FF5827404121E2874AF
:10246C00C72FF5827403121EB774212FF5827404E2
:10247C00121E2874512FF5827403121EB774AB2FE1
:10248C00F5827403121E28746D2FF5827403121ECC
:10249C00B774C72FF5827403121E28121EC0121DAA
:1024AC00F8FF900D86122003EB25E0FBEA33FA745B
:1024BC009C2BF58274053A121DF8FFE4FCFD900D7F
:1024CC008A1217CC900D8612177F74512BF58274DB
:1024DC00033AF583EEF0A3EFF0900D8A12177FAD5F
:1024EC0007AC06121DB6746D2FF5827403121E28EC
:1024FC00900D8A12177F900D8612201C12160890D0
:10250C000D8E1217CC900D8E121F72500302269155
:10251C00900D9812177F900D9412201C1216089093
:10252C000D801217CC900D80121F72500302269151
:10253C00900D9412177F780C12176C900D80121757
:10254C008B1257C5121F0E900D7FE0FF640B6004B9
:10255C00EFB4180C900D927404F0A374CBF0800AB5
:10256C00900D927403F0A37432F0900D92E0FEA3E0
:10257C00E0121EECD39FEC9E5009E4900D84F0A366
:10258C00F08015900D92E0FEA3E0FFC3ED9FFFECF1
:10259C009E900D84F0A3EFF0900D7FE0FF640B6034
:1025AC0004EFB4180F900D85E025E0F0900D84E059
:1025BC0033F08016900D84E0FEA3E0FF121ED212C1
:1025CC001F0E7D03121474121F0E900D7FE0121D4E
:1025DC00B71220743E121DF8121F4F900D84121F5B
:1025EC002CE4FCFD12205B900D7FE0121DB7122035
:1025FC0074121E281220743E121DF8FF900D84EEEA
:10260C00F0FCA3EFF0FD7B907A01900D7EE0F912C7
:10261C001DB712207C3E121DF8C39DEE9C5011126A
:10262C001EED121DB612207C121DA7121FFB802757
:10263C00121DB6121FFB3E121DF8121EECC39FECAE
:10264C009E5017121DB6121FFB121E28ED2BFDEC0F
:10265C003A121DB512207C121E28900D7EE0FD1240
:10266C001DB7121FFB3E121DF8FF121F0ED394FF55
:10267C00EE940F400A900D84740FF0A374FFF09049
:06268C000D84121FC022A4
:10382200900D70EFF0AF05EF121DB8121EC0F583B8
:10383200E0FFA3E0900D7CCFF0A3EFF0AF03EF1217
:103842001DB8121EC0121DF8FF900D7DE02FFF90D3
:103852000D7CE03EFEE4FCFD900D7E1217CCE47F71
:103862001EFEFDFC900D7E121F79500302392C9032
:103872000D7CE0FEA3E0FFE4FCFD780C12176CA3C4
:1038820012178B1257C5900D78122003900D7812E3
:10389200177F780C12176C900D781217CC1220300B
:1038A2007802C333CE33CED8F91220B312177FE495
:1038B2007B3F121F557806121759C004C005C00677
:1038C200C007900D7812177F7806121759D003D0CF
:1038D20002D001D000121608900D741220BDC0044F
:1038E200C005C006C0071220307802C333CE33CEE3
:1038F200D8F91220B3D007D006D005D0041220BDCB
:10390200E42FFFEE3408FEE43DFDE43CFC780C12AB
:103912001759D3EF94FFEE940F40047E0F7FFF9070
:0B3922000D70121E42A60608A6072228
:105D6B007C007D0B121462EEA2E713FEEF13FFC350
:105D7B0094CBEE648094845005E4FEFF8008743568
:075D8B002FFF74FB3EFE2216
:1058C500900D83ECF0A3EDF0121FD1125D6B121F4A
:1058D500D1121F173E121DF8121F4F900D81121F76
:1058E5002CEE3395E0FDFC12205B121F17121E28CB
:0C58F500121F243E121DF8FF121FD122CA
:10420900900D7EEFF0A3ECF0FEA3EDF0FFAC02AD54
:10421900031258C5900D7FEEF0FCA3EFF0FD7B2C47
:104229007A01900D7EE0F9121DB71220843E121D0D
:10423900F8C39DEC6480F8EE6480985011121F80D9
:10424900121DB6122084121DA71220098028121DE2
:10425900B61220093E121DF8FF121F80C31220C694
:104269005017121DB6122009121E28ED2BFDEC3A2B
:10427900121DB5122084121E28900D7EE0FD121D1C
:10428900B71220093E121DF8FF900D7FEEF0A3EF43
:10429900F0D394FFEE6480948F400A900D7F740FE1
:0C42A900F0A374FFF0900D7F121FC022E4
:1042B500A907E4FBFAE9FD3395E0FCED25E0FFEC09
:1042C50033FE12203BF583E020E403024353121F23
:1042D500B55025E964809498501EED25E0FFEC3338
:1042E500FE749C2FF5827405121EB7121EC0121D96
:1042F500F82DFFEE3CFE800A121DB6121EC0121DDF
:10430500F8FF125D6BAA06AB07121DB674162FF5E2
:104315008274053E121DF8D39BEE9A50317C007DC8
:1043250005AF03AE02121462AA06AB07EAC313FA7D
:10433500EB13FBD394FFEA940F40047A0F7BFFAD98
:1043450003121DB612203BF583EAF0A3EDF0AF0191
:0C435500EF121DB812203B121DF8FF22D1
:10290D00EF24FA900D76121E8E04900D7112204454
:10291D0070030229DC121F5B900D76121EF6900DCE
:10292D0070F0F470030229BFE0FF64117003022BF5
:10293D007FEF64127003022B7F121E6075F005EF9E
:10294D00121E4E7003022B7F90103BE0FF900D7412
:10295D00F0BF020B900D71E0FF900D70022A2890D0
:10296D000D74E0B40406900D70022A36900D74E0DB
:10297D0064036003022B7F900D701220AC5013EF97
:10298D009418500E121DDD900D72121EC9121FDA11
:10299D00800D900D70121F3AFFA3E0900D72CFF0D5
:1029AD00A3EFF0900D71122027900D70E0FB7A00CF
:1029BD00801A90103BE064036003022B7F900D7131
:1029CD00E0FF900D70E0FB7A00E4FDFC02420990FF
:1029DD000D76121E13900D76121F67E0900D75F097
:1029ED001260E5900D70EFF064117003022B7FE023
:1029FD00FF64127003022B7F121E6075F005EF123B
:102A0D001E4E7003022B7F900D71E0FF901023126C
:102A1D001E35E0900D74F0B40206A3E0FD0223CC48
:102A2D00121E79B40414900D75E0FF1242B5900D8D
:102A3D0071121E42A60608A60722121E79640360B3
:102A4D0003022B7F900D78F0A3F0A3F0A3F0900D6F
:102A5D0076E0900513121E17E4900D77F0900D7728
:102A6D00E0FFC3648094994003022B299005131253
:102A7D00182FEF3395E08F82F58374051218091224
:102A8D0013DF540F7003022B20900D77E0FD121D04
:102A9D00B7121EC0F583E0FFA3E0900D7CCFF0A32D
:102AAD00EFF0ED121FB65032900D77E0FF64809479
:102ABD00985027EF121DB8749C2FF58274053E12A5
:102ACD001DF8FF900D7DE02FFF900D7CE03EFE90F8
:102ADD000D72121ECE121FDA800B900D7CE0FFA33B
:102AED00E0900D72CFF0A3EFF0900D78E0FEA3E033
:102AFD00900D72122029D31220C64017900D78EC3C
:102B0D00F0A3EDF0900D77E0FE3395E0900D7AF0A7
:102B1D00A3CEF0900D77E004F0022A6A900D71E0DB
:102B2D00FF900D78E0FCA3E0FDA3E0FAA3E0FB121B
:102B3D004209300F3DE4900D77F0900D77E0FFC323
:102B4D00648094AD502AEF3395E0FE74FD2FF5822D
:102B5D0074143EF583E07010900D77E0121DB812DD
:102B6D001EC0F583E4F0A3F0900D77E004F080CA69
:032B7D00C20F2262
:10495400900D72121E882402900D71122044603250
:10496400121F5B900D73121EF6FFF4606D900D70B4
:10497400EFF0121E60900D70121E49605D121E5AF7
:10498400121EA6125781EF7802C333CE33CED8F964
:10499400803C900D73121E13900D73121F67E090EC
:1049A4000D72F01260E5900D70EFF0121E60900D24
:1049B40070E0121E4B6023900D72E0121E5B121EFB
:1049C400A6125781EF7802C333CE33CED8F9FF90C5
:0B49D4000D71121E42A60608A6072265
:103D7C00900D72121E882403900D71122044604F16
:103D8C00121F5B900D73121EF6FFF47003023E437C
:103D9C00900D70EFF0901043E064057027121E60D8
:103DAC00900D70121E497003023E43121E5A900071
:103DBC0003121EA9125781EF7802C333CE33CED82B
:103DCC00F9023E2B900D71E0FF900D70023E3E907B
:103DDC000D73121E13900D73121F67E0900D72F08D
:103DEC001260E5900D70EFF0121E60900D70E012F5
:103DFC001E4B6043900D71121E7C6405702E900D4D
:103E0C0072E0121E5BE92FF9EA35F0FA900003120A
:103E1C001EB0125781EF7802C333CE33CED8F9FFE0
:103E2C00900D71121E42A60608A60722900D71E095
:083E3C00FFA3E0FD1223CC22DC
:10470800900D70EFF0901022121E80900D74F01230
:1047180060E5900D73EFF0900D70E0FF121E7DB410
:104728000208900D74E0FD0223CC900D70121E7CDF
:10473800B4041B900D74E0FF900D73E06F70581275
:1047480042B5900D70121E42A60608A60722900DCB
:10475800741220AC5020EF9418501B121DDD900DE0
:1047680071121EC9900D71EEF0A3EFF00D121474C2
:10477800900D71EE800D900D74121F3AFFA3E0901A
:104788000D71CFF0A3EFF0900D70122027900D74EB
:08479800E0FB7A001242092245
:105781007B6A121F52900D741217CC900D74121770
:105791007FE47B64FAF9F81216A0900D741217CC0D
:1057A100E47FFF7E0FFDFC900D7412178BC312175F
:1057B10048400A900D741217D800000FFF900D7425
:0457C10012177F221A
:1061FA00781CE0FEA3E0A60608F62292AFAF028F53
:06620A00B1AF038F8422F6
:1051B500AB84AAB1A2AF9201900D5D1217CC900DF0
:1051C5005F1261FA53B10F900D5EE0700543B110A7
:1051D5008019900D5FE030E70543B130800D43B194
:1051E50020900D5FE04480F01261FAE4F584C2AFCF
:1051F50043B701758F03781CE6FE08E6F5828E83BA
:0D520500E4F053B7FEF58FA20112620522FE
:104E6600AB84AAB1A2AF9201900D691217CC900D36
:104E760068E0F9FF3395E0FEEFF44E6053900D6B5A
:104E8600781C1261FC53B10F900D6AE0700543B1B6
:104E9600108020900D6BE030E70543B1308014435D
:104EA600B120900D6BE04480F0E0FEA3E0781CA6F4
:104EB6000608F6E4F584C2AF43B701758F01781C86
:104EC600E6FE08E6F5828E83E9F053B7FEE4F58F39
:064ED600A2011262052298
:10347B00026E154A0270154A017407017207017634
:10348B0000016D005015370001FF00FF0000010126
:10349B000000FF00FF0100C115421535000041156A
:0234AB003400EB
:105B1600900D9F02182FD3ED9408EC648094802298
:105B2600D3ED9410EC6480948022C3ED94F8EC6479
:0E5B360080947F22C3ED94F0EC6480947F2273
:10503000900D9EEFF0E56F2401FFE4356EFAA907AD
:105040007B01A312184F125B1674019015CA6B7086
:1050500008E965827003EA6583700C7B017A157933
:105060004A900D9F12184F125B16EB8A8389826457
:1050700001700AE57165827004E5706583601990BE
:105080000D9EE0856F82856E83F0125B16AF018AFC
:095090006E8F6F900D9EE0F0227E
:105A1F0053E6F7E56FB57109E56EB57004E4FF80E5
:105A2F00210571E571AE707002057014F5828E83D9
:105A3F00E0FF74CAB5710B7415B5700675701575E6
:065A4F00714A43E6082243
:1060C80053E6F7E56FB57109E56EB57004E4FF8036
:0D60D80008857182857083E0FF43E6082291
:031A1E00022B8018
:102B8000C0E0C0F0C083C082C0D075D000C000C01B
:102B900001C002C003C004C005C006C007901428CD
:102BA000E06003022DA630DF02C2DFE5B05407F576
:102BB0007465726010E5746572F57675730355740B
:102BC000F56D857472E57360661573E5737060E585
:102BD00074540370069015347403F0E56D30E01AF8
:102BE000901534E0FE70047F01800CEE54FE9015C9
:102BF00034F030E1057F0D125030E56D30E11A9070
:102C00001534E0FE70047F02800CEE54FD90153404
:102C1000F030E0057F0D125030E57630E211E574BA
:102C200020E20C9015357401F0A374F4F0D2153045
:102C3000152E90153574FFF5F01214FF901535E040
:102C40007002A3E0700EC21590152AE0FF7D0412F9
:102C50005F56800CE5B030E207C2157F0412503099
:102C600020D90330D85BE5901313543F900D9CF0AE
:102C7000C2D8C2D9901549E0FF900D9CE0FD6F5479
:102C800003603EEF75F004A47E00540CFFED540386
:102C9000FDEF4D2437F582EE3415F583E0900D9D60
:102CA000F06016E0FF3395E09015478FF01214FFA7
:102CB000901532E4F0A37405F0900D9CE090154956
:102CC000F0901532E07002A3E0600A90153274FFB4
:102CD000F5F01214FF901532E07004A3E064016077
:102CE00003022DA6901547E0FCA3E0FD64024C70A2
:102CF000057F05022D9C125B1C50047F0180027F22
:102D000000901547E0FCA3E0FDD39402EC648094AE
:102D10008040047E0180027E00EE5F60057F070236
:102D20002D9C125B2650047F0180027F00125B1CE9
:102D300040047E0180027E00EE5F60047F09805CBB
:102D4000125B2640047F0B8053BCFF07BDFE047F4F
:102D5000068049125B3040047F0180027F00C3ED92
:102D600094FEEC6480947F50047E0180027E00EE2D
:102D70005F60047F088025125B3A40047F01800277
:102D80007F00125B3050047E0180027E00EE5F60A7
:102D9000047F0A8007125B3A500C7F0C125030906F
:102DA0001547E4F0A3F0D007D006D005D004D00337
:102DB000D002D001D000D0D0D082D083D0F0D0E0EB
:012DC00032E0
:10627900E475F00112151585F082F58322EEF0A37D
:04628900EFF0A3226D
:0B63CA00AF01AE027C00E4FD0251B503
:10622500900D63EDF0AF01AE027C00E4FDE0900D52
:0562350068F0024E6656
:10531E00900D5D126286ECF0A3EDF0A3EAF0A3EB24
:10532E00F0900D61E07002A3E0603A900D5DE0FE3A
:10533E00A3E0AA06F97B01A3E0FEA3E0F5828E832B
:10534E00E0FD126225900D6174FFF5F01214FF90CE
:10535E000D5FE475F0011214FF900D5DE475F00120
:06536E001214FF80BC22B6
:08641A00E49006CFF0A3F0228C
:105C22009006CFE0FEA3E0AA06F97BFF1263CA90BA
:105C320006CFE0FEA3E0FF7C067DD17B007A041252
:0A5C4200531EE49006CFF0A3F022F9
:104BEF00900D58EDF0900D56EEF0A3EFF0EE54FC53
:104BFF00FE9006CFE0FCA3E0FD7002EE6C6044ED8A
:104C0F004C6003125C22900D56E0FEEE54FCFE7FCA
:104C1F00009006CFF0A3EFF0900D59126286740644
:104C2F00F0A374D1F07FFF7E03900D59126279E4E7
:104C3F0093FD900D5B126279EDF0EF1F70011EEF87
:104C4F004E70E6900D58E0FF900D56E0FCA3E0FD8E
:104C5F00EC5403FC74D12DF58274063CF583EFF010
:014C6F002222
:1059B000900ADF12628612184F900AE474FFF5F025
:1059C00012151545F06020900ADFE475F0011215FC
:1059D00015AFF0FE900AE1E475F0011218381213C9
:0859E000C6FD124BEF80D2223C
:1053C9000001020408100000030418000000000096
:1053D9001F0000000000180403000000001008046A
:1053E90002010000040A0A11110000010102021C55
:1053F90000001C020201010000101008080700004B
:0E5409000708081010000020406080A0C0FFBF
:0E6364007F147E00EF1F70011EEF4E70F722B7
:1062F8007F381260307F061260307D0EE4FF026343
:01630800A6EE
:10603000900AE7EFF0A2AF9202C2AF125F36EF20F4
:0F604000E7F9900AE7E0FF12608DA20292AF220B
:105F3600A2AF9203C2AF75A0FFC2B5D2B6D2B71256
:105F46006364ADA0C2B7126364A20392AFAF052229
:0564A8007F01026030DD
:10608D00A2AF9203C2AF8FA0126364C2B5C2B6D2E3
:0E609D00B7126364C2B7126364A20392AF220B
:10611D00A2AF9203C2AF8FA0C2B6D2B7D2B51263EF
:0B612D0064C2B7126364A20392AF22A9
:0C63A600901607E05FF04DFFF002603041
:10616B00AC07A2AF9202C2AF125F36EF20E7F9AFD6
:09617B000412611DA20292AF2280
:105DE000900AE712184F900AE712182F1213C66094
:105DF00013900AE7E475F0011218381213C6FF1267
:055E0000616B80E2224D
:10597600900AE112184FA2AF9201C2AF1264A8E4D6
:10598600FDFF1263B2900AE112182F125DE0E4FDEA
:105996007F011263B2900AE412182F125DE07D10A7
:0A59A6007F011263B2A20192AF224A
:0C63B200EF75F040A42D2480FF02603045
:0B63D500E4F584EF90540F93F5D32201
:1044A100900AE0EDF0900ADD12184FAF01900AE595
:1044B100EAF0A3EFF0900AE174FF121799EC4D4E68
:1044C1004F6078900ADD12182FE92428F9E43AFAAE
:1044D100C003C002C001900AE5E0FEA3E0FFF9D0ED
:1044E10082D083D0E064017008E965827003EE65D3
:1044F100836020900ADD12182FE92442F9E43AFA88
:10450100EB8A83898264017008EF65827003EE652E
:104511008370098F828E837404F08012900AE0E028
:10452100FF900AE5E0FCA3E0F5828C83EFF0900AAE
:0C453100E5E475F0011214FF0244B6220C
:105F5600900D9EEFF0A3EDF07F0A125212900D9E67
:105F6600E0FF125212900D9FE0FF1252120263726E
:086422007F02125212026372A4
:105AB80012646FEF6027900ADB7416F0A37400F08D
:105AC800125D1B900ADBE475F00112151585F08252
:105AD800F583EFF0126475EF70E67F01227F0022F4
:10623A00900ADBEFF07F2F125212900ADBE0FF1276
:05624A00521202637214
:10624F00900ADBEFF07F30125212900ADBE0FF1260
:05625F005212026372FF
:10392D0090700175F070ED12181AEC75F070A425F9
:10393D0083F8ED25E028AF82900AE7F0A3EFF09031
:10394D000ADFE0FF7E007C027D7012146274012F8D
:10395D00F974703EFA7BFF22E0FF75F070907001F4
:10396D0012181AEF25E02583AF8222900D53E475CE
:10397D00F0010214FFFE7A10792074027B01900A87
:10398D00E4F0A322900ADCE475F001121838AE02BF
:10399D00AF0122E024FFFFE434FFFE900AE0E0FCDB
:1039AD00A3E0FD22900D53E0FCA3E0FDC39470EC69
:1039BD00940222E475F00112151585F082F583E469
:1039CD00932224FFFEE434FF900AE0F0A3CEF02210
:1039DD00900AE412184FE4900AE2F0A3F022AD042D
:1039ED00EDFFEEF0A3EFF022E4900D53F0A3F022E3
:1039FD00AF05E4F0A3EFF0E07F00FE2274E12DF5BA
:103A0D0082740A3CF583229FEE6480F8EC64809802
:013A1D002286
:10537400900ADB7402F0E4A3F012641A7E707F00DA
:105384007A0A79DBE412398904F01259B07EBB7FC2
:10539400917B017A0A79DC900AE4E4F0A304F01228
:1053A40059B0125C227B017A107920900AE112171D
:1053B400D800000270E4FD1244A112453D1261B50B
:0553C4007F1E025901EB
:1061840090BB91E493600C907000E493640260030C
:09619400125374E490101EF02275
:10590100900ADDEFF012641AE4900ADEF0900ADDED
:10591100E0FFA3E0FEC39F501F75F070EE90700191
:1059210012181AEE1239711239827470F01259B0CC
:0B593100900ADEE004F080D5025C224A
:1062B10030110920170B126422D21722D210123A80
:0262C1001E229B
:031A1B000262B1B3
:1059E800900ADC12184F900AE274FFF5F0121515B0
:1059F80045F06022900ADF12182F1213C6FF900A92
:105A0800DC12182FEF12142E900ADD12397B900A3F
:075A1800E012397B80D0226F
:105C4C00901022E0900ADBF090101E12394F900A4F
:105C5C00DF12184F900AE27402F0A37470F07B010B
:0A5C6C007A1079201259E8C21722BD
:1062640012641A90101E1239651239827470F01279
:0562740059B0025C229C
:1061B500A2AFE433900ADDF0C2AF126264C2179059
:0861C5000ADDE024FF92AF2285
:103BE700900ADBEFF0A3EDF0A2AFE433900AE9F01F
:103BF700C2AF900ADBE0FFD39B4033EF1239CFEB24
:103C070014900ADFF0900ADC1239A0D3123A14504C
:103C17005812392D1239DD123C7940FB125C229083
:103C27000AE012397B900ADFE004F0023C0C900AAC
:103C3700DCE01239CF900ADEE014A3F0900ADB1221
:103C470039A0C3123A14402112392D1239DD123C22
:103C57007940FB125C22900AE074FFF5F01214FF22
:103C6700900ADFE014F0023C43900AE9E024FF9257
:103C7700AF22900AE4E475F001121838AE02AF01E2
:103C8700900AE7E475F00112151585F082F583E4D3
:103C970093FD124BEF900AE2E475F0011214FFC393
:0D3CA700900AE3E09470900AE2E09402229B
:103E4400900ADBEDF0A2AFE433900D55F0C2AFEF72
:103E540014900D51F0EB14A3F0900ADBE014FF90E2
:103E64000D51E0D39F4003023F03A3123965FE12B4
:103E740039F51239B150190FEFAA0670010E14F575
:103E8400828A83E493FB123A09EBF012397880E2D8
:103E9400900D5212394F900ADC12184F900D5112A6
:103EA4003965900ADFF0A3EFF01239F512399190D9
:103EB4000ADF1239C0FD124BEF123978C3900D544A
:103EC400E09470900D53E0940240E1900D5112394A
:103ED4004F900ADC12184F1239F51239B1501012F2
:103EE4003991123A09E0FD124BEF12397880EB1246
:103EF4005C22900D51E004F0A3E004F0023E5D90DA
:083F04000D55E024FF92AF22ED
:1047A000900ADBEBF0AC07A31239FD900ADCF0A312
:1047B000EFF0900ADC1239EBA2AFE433900AE5F097
:1047C000C2AF900AE4740FF012641A900AE412392E
:1047D0004F900AE012184FE4900ADEF0A3F0900A1E
:1047E000DCE0FCA3E0FFECFD900ADBE0FBE4900AD8
:1047F000E9F0D201123B07900AE3EFF0FD900AE0E6
:10480000123994124BEF900ADC12397B900ADE12B7
:10481000397BC3900ADFE09470900ADEE094024096
:10482000BD125C22900AE4E004F0E0C3941E4098BC
:08483000125888D2AF0264089F
:1045D700900ADBEBF0AC07A2AFE433900AE3F0906C
:1045E7000ADE1239FD900ADEF0A3EFF0900ADE1220
:1045F70039EBC2AF900AE2740FF0900AE2E0FFC312
:10460700941E505675F070EF12396A900AE0F0A3C5
:10461700EFF0E4900ADCF0A3F0900ADEE0FCA3E000
:10462700FFECFD900ADBE0FB900AE01239C0900A2C
:10463700E9F0C201123B07900ADE12397B900ADCCF
:1046470012397BC3900ADDE09470900ADCE0940293
:1046570040C7900AE2E004F080A01264081258886C
:09466700900AE3E024FF92AF2267
:103B0700900AE6EFF0A905C20220C3FD20C5FAC25C
:103B1700C4D2C5E4FFFD30C3FD30C3FDE5C154F891
:103B2700FC64086004ECB41013EFB40105EB440126
:103B37008003EB54FEF5C27D01023BD5ECB4180BB4
:103B470089C27D02C2C4C2C5023BD5ECB420028043
:103B570045EC6428703CEDB4020E900AE6E0F5C22D
:103B67007D03C2C5C2C48066EDB4031B300108D211
:103B7700C57F01C2C48057900AE9E0F5C2C2C57D7E
:103B870004E4FFC2C48047ED64047042D2C47D05DB
:103B9700803CECB4300AD2C4D2C57D08E4FF802E45
:103BA700ECB438028024ECB44006C2C2C2C5801E01
:103BB700ECB448028014ECB450028004ECB4580A08
:103BC700D2C47D07AEC2C2C28004D2C4D2C5C2C3AA
:103BD700ED64076008ED64056003023B20AF062231
:105C76007E0E7F8E8E648F658E608F617E0F7F565F
:105C86008E668F678E628F63E4F56CC21B7E0D7F16
:0A5C9600A38E6A8F6B8E688F69225F
:031A0F00024FC1C2
:104FC100C0E0C083C082C0D0309821C29885618280
:104FD100856083E599F00561E56170020560B4566D
:104FE1000BE560B40F0675600E75618E309937E57B
:104FF1006C602F856782856683E0900DA2F0C2996F
:10500100F599900E6BE599F0156C0567E5677002EF
:105011000566B41E11E566B4100C75660F7567560A
:0F5021008004C299C21BD0D0D082D083D0E0329D
:1062C300E56165657004E560656460037F01227FB5
:0262D3000022A7
:10604F00856582856483E0FF0565E56570020564FB
:0F605F00B4560B740FB5640675640E75658E220A
:031A3F000256B498
:1056B400C0E0C083C082C0D030982CC29885698273
:1056C400856883E599F0E0648E600690152E740772
:1056D400F00569E56970020568B46B0BE568B40E02
:1056E4000675680D7569A3309902C299D0D0D0822D
:0556F400D083D0E0327C
:1062D500E569656B7004E568656A60037F01227F87
:0262E500002295
:10606E00856B82856A83E0FF056BE56B7002056ABE
:0F607E00B46B0B740EB56A06756A0D756BA322B1
:0A34AD004115D2004115EB00C11AD1
:105809009015D5E475F00112151585F082F58322FE
:105819009015D57415F0A374ECF0229015CCE475AD
:10582900F0011214FF7E167F009015CCE02290152E
:10583900D0E0FFA3E09015CC22E0F5C29015CCE0B2
:025849006E22CD
:10610100AF84E4F584C2C343E60243F60275C301DA
:0C61110075C04475CF8F43C3018F8422FA
:105888007E157FD79015CEEEF0A3EFF09015D3EEEE
:10589800F0A3EFF09015CAEEF0A3EFF07E157FECC1
:1058A8009015D0EEF0A3EFF09015D5EEF0A3EFF041
:0D58B8009015CCEEF0A3EFF0C219026101D3
:105D92009015D312580CEFF09015D312580CEDF069
:105DA2009015D3E0B4150FA3E0B4EB0A9015D374A9
:075DB20015F0A374D7F022E5
:0E637200AF84E4F584C219C2C4D2C58F842260
:1052120020192FD21912580974FFF07C167D0090C4
:1052220015D5E0B50408A3E0B505031258191258C4
:1052320009E4F09015D5E0B50408A3E0B505031222
:105242005819125809E4F09015D5E0B41608A3E0F5
:10525200B40003125819125809EFF09015D5E0B4B2
:0D5262001608A3E0B400031258197F0122C2
:105BF6009015CEE0FCA3E0FD9015CAE0B50408A31D
:105C0600E0B505037F00229015CEE0FCA3E0F58207
:0C5C16008C83E0B507037F01227F002291
:105D1B009015CEE475F0011214FF9015CE12580CAD
:105D2B00E0FF9015CEE0B4150FA3E0B4EB0A90158D
:095D3B00CE7415F0A374D7F02218
:06646F007FFF125BF62224
:06647500E4FF125BF622B9
:031A1800022FFF9B
:102FFF00C0E0C0F0C083C082C0D075D000C000C098
:10300F0004C005C006C007E5C154F8121884316723
:10301F0000305A08305A1030831830AA2030B028A8
:10302F00311230311738312150312158312D603163
:10303F002368312D70312378312180313C88312143
:10304F0090313C98314FA000003194C2C5125824E2
:10305F00B5060BA3E0B507069015CC12581C9015BA
:10306F00CC12580C1258427003A3E06F6003023168
:10307F0094023109125824B5060BA3E0B507069048
:10308F0015CC12581C9015CC12580C1258427003C4
:10309F00A3E06F6003023194023109125837CF80D9
:1030AF001B9015D5E0FEA3E0FF9015CCE0FCA3E04C
:1030BF00FDB50713ECB5060F9015D0EEF0A3EFF0AA
:1030CF00C2C5D2C40231948D828C83E0B4FF07C293
:1030DF00C4D2C5023194125824B5060BA3E0B5072C
:1030EF00069015CC12581C9015CC12580C12584241
:1030FF007003A3E06F60030231949015CC12581C3B
:10310F00023194125837802F125837CFF0A3EFF0B7
:10311F0080738010125837CFF0A3EFF0D21AADC2E0
:10312F007FFF8004ADC2E4FF125D9280589015CAF4
:10313F00E0FFA3E09015D3CFF0A3EFF0D2C480450A
:10314F009015D3E0FFA3E09015CACFF0A3EFF030B6
:10315F001A33D2C5C21A802D9015D0E0FEA3E0FF1E
:10316F009015CCEEF0A3EFF09015CAE0FDA3E09020
:10317F0015D3CDF0A3EDF0D2C4A3E06E7003A3E09E
:10318F006F6002D2C5C2C3D007D006D005D004D01D
:0C319F0000D0D0D082D083D0F0D0E0323D
:100C1A00020C9AE493A3F8E493A34003F68001F24A
:100C2A0008DFF48029E493A3F85407240CC8C333DB
:100C3A00C4540F4420C8834004F456800146F6DFAA
:100C4A00E4800B0102040810204080903353E47EB4
:100C5A00019360BCA3FF543F30E509541FFEE4939F
:100C6A00A360010ECF54C025E060A840B8E493A366
:100C7A00FAE493A3F8E493A3C8C582C8CAC583CA91
:100C8A00F0A3C8C582C8CAC583CADFE9DEE780BE49
:0134B7000014
:1013C600BB010689828A83E0225002E722BBFE0225
:0913D600E32289828A83E4932258
:1013DF00BB010CE58229F582E5833AF583E02250C3
:1013EF0006E92582F8E622BBFE06E92582F8E2220D
:0D13FF00E58229F582E5833AF583E4932227
:10140C00BB010989828A83F8E028F022500327F770
:10141C0022BBFE05F8E328F3228A838982F8E49341
:02142C00282274
:10142E00BB010689828A83F0225002F722BBFE019D
:02143E00F32297
:10144000F8BB010DE58229F582E5833AF583E8F0E2
:10145000225006E92582C8F622BBFE05E92582C88E
:02146000F22276
:10146200EF8DF0A4A8F0CF8CF0A428CE8DF0A42E9E
:02147200FE2258
:10147400BC000BBE0029EF8DF084FFADF022E4CC5C
:10148400F875F008EF2FFFEE33FEEC33FCEE9DEC25
:10149400984005FCEE9DFE0FD5F0E9E4CEFD22ED6B
:1014A400F8F5F0EE8420D21CFEADF075F008EF2FB5
:1014B400FFED33FD4007985006D5F0F222C398FDA6
:0514C4000FD5F0EA2243
:1014C900C2D5EC30E709B2D5E4C39DFDE49CFCEE3E
:1014D90030E715B2D5E4C39FFFE49EFE121474C32E
:1014E900E49DFDE49CFC800312147430D507C3E429
:0614F9009FFFE49EFE22AD
:1014FF00C5F0F8A3E028F0C5F0F8E5821582700278
:06150F001583E038F02214
:10151500A3F8E0C5F025F0F0E58215827002158389
:06152500E0C838F0E822E6
:10152B00BB010A89828A83E0F5F0A3E0225006878B
:10153B00F009E71922BBFE07E3F5F009E31922894D
:0B154B00828A83E493F5F07401932280
:10155600BB0110E58229F582E5833AF583E0F5F0D3
:10156600A3E0225009E92582F886F008E622BBFEB0
:101576000AE92582F8E2F5F008E222E5832AF583F6
:08158600E993F5F0A3E99322BB
:10158E00BB010DC58229C582C5833AC5830214FFEE
:10159E005011C58229F808E5F026F618F5F0E58217
:1015AE0036F622BBFE11C58229F808E225F0F5F0C9
:1015BE00F218E23582F222F8E58229F582E5832AD5
:0D15CE00F58374019325F0F5F0E4933822C5
:1015DB00F8BB0111E58229F582E5833AF583E8F042
:1015EB00E5F0A3F0225009E92582C8F608A6F022FF
:0D15FB00BBFE09E92582C8F2E5F008F222E6
:0D160800EF2BFFEE3AFEED39FDEC38FC2231
:10161500E88FF0A4CC8BF0A42CFCE98EF0A42CFC74
:101625008AF0EDA42CFCEA8EF0A4CDA8F08BF0A4F2
:101635002DCC3825F0FDE98FF0A42CCD35F0FCEB51
:101645008EF0A4FEA9F0EB8FF0A4CFC5F02ECD3916
:0F165500FEE43CFCEAA42DCE35F0FDE43CFC2283
:1016640075F008758200EF2FFFEE33FECD33CDCC3D
:1016740033CCC58233C5829BED9AEC99E5829840C0
:101684000CF582EE9BFEED9AFDEC99FC0FD5F0D69D
:10169400E4CEFBE4CDFAE4CCF9A88222B800C1B9C7
:1016A4000059BA002DEC8BF084CFCECDFCE5F0CB05
:1016B400F97818EF2FFFEE33FEED33FDEC33FCEB3E
:1016C40033FB10D703994004EB99FB0FD8E5E4F9F9
:1016D400FA227818EF2FFFEE33FEED33FDEC33FCE6
:1016E400C933C910D7059BE99A4007EC9BFCE99ADA
:1016F400F90FD8E0E4C9FAE4CCFB2275F010EF2F1F
:10170400FFEE33FEED33FDCC33CCC833C810D7071E
:101714009BEC9AE899400AED9BFDEC9AFCE899F859
:0E1724000FD5F0DAE4CDFBE4CCFAE4C8F922EC
:1057C500C2D5E830E70FB2D5E4C39BFBE49AFAE40F
:1057D50099F9E498F8EC30E717B2D51257FB121691
:1057E500A0E4C39BFBE49AFAE499F9E498F88003F2
:1057F5001216A030D50DE4C39FFFE49EFEE49DFD87
:04580500E49CFC2201
:10173200EB9FF5F0EA9E42F0E99D42F0EC6480C82E
:0617420064809845F022CE
:10174800EB9FF5F0EA9E42F0E99D42F0E89C45F0F7
:01175800226E
:10175900E8600FECC313FCED13FDEE13FEEF13FF6E
:03176900D8F12292
:10176C00E8600FEFC333FFEE33FEED33FDEC33FCDB
:03177C00D8F1227F
:0C177F00E0FCA3E0FDA3E0FEA3E0FF22DD
:0C178B00E0F8A3E0F9A3E0FAA3E0FB22E1
:101797007401FF3395E0FEFDFCA3A3A3E0CF2FF078
:1017A700E582158270021583E0CE3EF0E582158250
:1017B70070021583E0CD3DF0E58215827002158336
:0517C700E0CC3CF02223
:0C17CC00ECF0A3EDF0A3EEF0A3EFF02290
:1017D800A8828583F0D083D0821217EF1217EF12F8
:1017E80017EF1217EFE473E493A3C583C5F0C5831D
:1017F800C8C582C8F0A3C583C5F0C583C8C582C85B
:0118080022BD
:10180900F5F0C582A4C582C5F0C583A42583F583F7
:0118190022AC
:0C181A00A42582F582E5F03583F58322D9
:09182600E6FB08E6FA08E6F922E7
:09182F00E0FBA3E0FAA3E0F922BA
:10183800F8E0FBA3A3E0F925F0F0E5821582700239
:071848001583E0FA38F022DD
:09184F00EBF0A3EAF0A3E9F0229A
:0C185800E493FB740193FA740293F922EC
:10186400BB010789828A8302182F5005E9F8021800
:1018740026BBFE05E9F80218B089828A830218584B
:10188400D083D082F8E4937012740193700DA3A3F3
:1018940093F8740193F5828883E473740293686007
:0618A400EFA3A3A380DF07
:0618AA008A838982E473C9
:101A4200E51724E4F582E4340AF583E005172290D1
:101A52000AE1300803900AE4E475F0011218380232
:101A620013C62001E97F2ED2018018EF540F249073
:101A7200D43440D4FF30050BEF24BFB41A00500316
:101A82002461FFE51860021518051BE51B700205AD
:101A92001A30080E900AE1E475F001121838EF02CC
:101AA200142E025DB97403D2088003E4C208F5174C
:101AB200900AE112184FE4F518F51AF51BE51860C3
:101AC200077F20121A8580F57519FFC202C201C272
:101AD20003C204C206C207C209121A51FF700D30B6
:101AE20008057F00121A96AF1BAE1A22B4255FC2F8
:101AF200D5C205121A51FF24D0B40A00501A75F04B
:101B02000A781830D50508B6FF0106C6A426F620C5
:101B1200D5047002D20480D924CFB41A00EF500445
:101B2200C2E5D205021C97D20280C6D20180C0D281
:101B32000380BCD2D580BAD20680B47F20121A8527
:101B42002003077401B5180040F1121A42FF121A5D
:101B520085021ABFD209D2078095121A42FB121AC5
:101B620042FA121A42F94A4B700679687A1D7BFFD3
:101B720020032EE518602A7E008E827583001213E0
:101B8200DF60060EEE651970F0C2D5EBC0E0EAC068
:101B9200E0E9C0E0EE121CDED0E0F9D0E0FAD0E0DD
:101BA200FB1213C6FF60AAEBC0E0EAC0E0E9C0E0A6
:101BB200121A85D0E02401F9D0E03400FAD0E0FB1B
:101BC200E5190460DCD519D980877BFF7A1C79DAA4
:101BD200D203809C791080027908C207C20980086A
:101BE200D2D5790A8004790AC2D5E519047002F5C2
:101BF20019E4FAFDFEFF121A42FC7B0820021312BE
:101C02001A42FD7B1030010A121A42FE121A42FFDA
:101C12007B20EC3382D592D55013C3E43001069F6A
:101C2200FFE49EFEE42002039DFDE49CFCE4CBF86D
:101C3200C202EC700CCFCECDCCE824F8F870F38061
:101C420017C3EF33FFEE33FEED33FDEC33FCEB3322
:101C5200FB994002FB0FD8E9EB300205F8D0E0C453
:101C620048B202C0E00AEC4D4E4F78207B0070C2B1
:101C7200EAB5190040BCC0E0121CE0D0F0D0E02070
:101C82000204C4C0E0C4B202C0F0121A6ED0F0D591
:101C9200F0EB021ABF1218841B5C531BD6581B2D83
:101CA2004C1B29421BDA4F1BE2441BE2491B4243F5
:081CB2001BE8551BCC461BCCBE
:101CBA00451BCC471D88501B312D1B352E1B582B1D
:101CCA001B39231B56201D712A1AF14800001B508C
:101CDA003F3F3F00790AA2D5200414300609B91003
:101CEA00020404B9080104A2D52007025001042005
:101CFA0003689203B518005034C0E07F20300419FD
:101D0A007F30A20372077206500F121D37C203C238
:101D1A0007C206C2097F30800F300603E9C0E0120D
:101D2A001A85300603D0E0F9D0E0B518CC30061792
:101D3A007F30B9100C121A857F583005077F7880DA
:101D4A0003B90803121A853003057F2D021A857F0D
:101D5A00202009F87F2B2007F322920380CF286ED8
:101D6A00756C6C2900D202121A423002F8C202784B
:101D7A001830D50108F6021AF12D50434958121AA3
:101D8A00422403B405004001E4901D8393121A769D
:0D1D9A00743A121A76D204751804021BD692
:0C63BE00EE30E707C3E49FFFE49EFE22E0
:0918B000E2FB08E2FA08E2F92269
:105DB900EFB40A07740D125DC4740A309811A899DA
:105DC900B8130CC2983098FDA899C298B811F6304A
:075DD90099FDC299F5992222
:00000001FF
